:020000040800F2
:100000005809002045010008BD100008251000080F
:10001000B9100008B1010008D32D0008000000004D
:10002000000000000000000000000000952400080F
:10003000B50D00080000000035200008E12600088A
:100040005F0100085F0100085F0100085F01000810
:100050005F0100085F0100085F0100085F01000800
:100060005F0100085F0100085F0100085F010008F0
:100070005F0100085F0100085F0100085F010008E0
:100080005F0100085F0100085F0100085F010008D0
:100090005F0100085F0100085F0100085F010008C0
:1000A0005F0100085F0100085F0100085F010008B0
:1000B0005F010008492700085F0100085F01000890
:1000C0005F0100085F0100085F0100085F01000890
:1000D0005F0100082929000885290008692A00080D
:1000E0005F0100085F0100085F0100085F01000870
:1000F0005F0100085F0100085F0100085F01000860
:100100005F0100085F0100085F0100085F0100084F
:100110005F0100085F0100085F0100085F0100083F
:100120005F0100085F0100085F0100085F0100082F
:10013000DFF80CD000F02AF800480047D92E00085C
:10014000580900200648804706480047FEE7FEE7BA
:10015000FEE7FEE7FEE7FEE7FEE7FEE7FEE7FEE777
:10016000E526000831010008D2B201E000F8012BB9
:10017000491EFBD270470022F6E710B513460A4627
:1001800004461946FFF7F0FF204610BD064C074D08
:1001900006E0E06840F0010394E807009847103457
:1001A000AC42F6D3FFF7C8FFF03100081032000868
:1001B00000BFFEE710B502460B460020002104E018
:1001C000545C0444E0B24C1CE1B29942F8DBC443F5
:1001D000E0B2441CE0B210BDFEB5002000900190DA
:1001E000029000F039FF414800780A281DD14048AC
:1001F000007840490978884217D13D4840783D4908
:100200004978884211D13A48007A3A49097A8842B5
:100210000BD13748407A3749497A884205D1364868
:10022000008840F40040344908803348008800F4D6
:100230000040002858D0012002F0FAFD00202F498C
:10024000087048708870C87008712D49087048702F
:100250008870C87008712B49087048708870C87021
:1002600008712949087048708870C870087100F0DA
:10027000F3FE0020224908701D48007948701C4890
:10028000407988701A488079C8701948C079087117
:1002900000201E4908701A48407848701848807835
:1002A00088701748C078C870154800790871012017
:1002B00001F0A8F912484078040611488078050436
:1002C0000F48C0780602601930440D490979471873
:1002D00001200F49087000F0BFFE00F0BDFE0020B5
:1002E0000249087004490880FEBD00000900002092
:1002F000CC0100200C0000200A0000202C0000206F
:100300001600002034000020390000201B000020CF
:100310004100002010B588B07F480078012838D10E
:1003200000207D490870FC207C490870112048702D
:100330007B48007888707A484078C8707848807820
:1003400008717748C078487175480079887107212D
:100350007248FFF72FFF7149C8710020714908608A
:10036000FF22E121012001F0B3FD08236B4AA821FF
:10037000012001F06FFD012001F044F901206A49DC
:10038000C1F8A4016949087000206949088000F09B
:1003900063FE6748008840F6B83188427BDC00F095
:1003A0005BFE604884380068002857D100F054FE96
:1003B0006946012001F02CFD0446204602F0B8F801
:1003C0005CA002F0BFF804F040004028EDD100200E
:1003D0008DF80A000721684600F0EDFC55A002F0F8
:1003E000B1F89DF801004E490978884254D19DF832
:1003F00002004B49497888424ED19DF80300484994
:100400008978884248D19DF804004549C9788842D6
:1004100042D19DF805004249097988423CD14348C0
:10042000007801281BD141480078401C3F490870E2
:1004300012203A49487007213848FFF7BBFE374978
:10044000C8710020374908600823344AA8210120D8
:1004500001F000FD01203449C1F8A40158E000205A
:10046000324908700E21344800F0A5FC31A002F09A
:1004700069F832480178012001F01EF910202E4958
:1004800048700E212C4802F047F82DA002F05AF8CF
:10049000012008B010BD16E000202249086011209C
:1004A0001E49487007211D48FFF784FE1B49C8718B
:1004B00008230A46A821012001F0CCFC01201A499A
:1004C000C1F8A40124E00020154908704870887024
:1004D000C87008711B49087048708870C87008712E
:1004E0001949087048708870C870087117490870F9
:1004F00048708870C870087130200F4948700E210C
:100500000D4802F009F812A002F01CF80120C0E723
:1005100000F0A2FD0020BCE73E00002042000020C9
:100520002C000020A4812142008021428200002072
:10053000200000200A000000C00300202A00002044
:100540004F4B0A00390000201B000020160000203D
:10055000333030300A00000010B588B03F480088C2
:1005600040F2DC5188426DDA3D480068002866D1CF
:1005700000F072FD6946012001F04AFC044604F0D7
:10058000400040285BD100208DF80A000721684612
:1005900000F011FC33A001F0D5FF9DF8010078B9FF
:1005A0009DF8020060B99DF8030048B900202E496B
:1005B000087048708870C8700871012008B010BDBC
:1005C0002A480078072803D0284800780D280FD142
:1005D0000020254908709DF8000048709DF8010032
:1005E00088709DF80200C8709DF80300087124E02F
:1005F0001E480078082810D19DF801001A4908709B
:100600009DF8020048709DF8030088709DF8040072
:10061000C8709DF8050008710FE09DF805001249AB
:1006200008709DF8010048709DF8020088709DF8E0
:100630000300C8709DF8040008710120BEE700F0B7
:100640000BFD08E000200849087048708870C870E9
:1006500008710120B2E70020B0E70000320000205E
:10066000208121420A000000390000202A000020D9
:1006700010B500F0F1FCFE480078082829D1FD48AB
:100680000078752825D1FB484078702821D1F94899
:10069000807864281DD1F748C078612819D1F548C1
:1006A0000079742815D1F3484079652811D10020CC
:1006B000EF49087000BFF048006800F4E060EF49BF
:1006C0000843001DEC490860BFF34F8F00BF00BF17
:1006D000FEE7E8480078752807D0E6480078FA2851
:1006E00003D00020E249087010BDE14800780E28D0
:1006F00000DAF9E7DE480078401EDE49085CFB2896
:1007000000D0F1E7DB48807AA02804D1D8480078EF
:10071000152800D0E8E7D64800780E281ED1D54825
:100720000078FA2814D1D348407BFB2810D1D44854
:10073000008840F40040D24908800020CC4908706D
:100740000E21CC4800F037FBCEA001F0FBFE4AE0C2
:100750000020C7490870CA49088044E0C4480078AE
:1007600015281ED1C3480078FA2814D1C148007D4D
:10077000FB2810D1C248008840F40040C0490880DE
:100780000020BB4908701521BA4800F014FBBDA039
:1007900001F0D8FE27E00020B5490870B84908806C
:1007A00021E0B348007811281DD1B2480078FA281A
:1007B00014D1B048007CFB2810D1B148008840F427
:1007C0000040AF4908800020A94908701121A948BC
:1007D00000F0F1FAABA001F0B5FE04E00020A4495E
:1007E0000870A7490880A648008800F40040002847
:1007F00071D000F031FC9F488079A34988719D48F1
:10080000C179A148C1719B48017A9F4801729948FA
:10081000417A9D4841729748807A9B498872084680
:1008200080799A4988719848C1799848C1719648E9
:10083000017A964801729448417A944841729248EC
:10084000807A94284CD018DC732834D00CDC25280E
:1008500025D004DC21281AD022287DD11BE02628AF
:1008600021D07128F9D122E0742828D075282AD007
:1008700078282CD08228F0D12EE0A03809286BD21D
:10088000DFE800F0329CA0F5F4F3F2F1F000002074
:100890007D498872CBE100207B498872C7E1002046
:1008A00079498872C3E1002077498872BFE100204E
:1008B00075498872BBE1002073498872B7E1002056
:1008C00071498872B3E100206F498872AFE100205E
:1008D0006D498872ABE1AEE100206B498872A6E1F8
:1008E000002069498872A2E10020614908706648C9
:1008F0008079674988716448C1796548C1716248E7
:10090000017A634801726048417A614841725E48E9
:10091000807A5F4988725748407B5B4948735548E5
:10092000817B594881735348C17B5748C1735148F3
:10093000017C554801744F48417C534841744D48EF
:10094000407B544908704B48807B48704948C07BC5
:1009500088704848007C00E068E1C8704548407CE9
:10096000087101204C49087000204C490880012082
:1009700000F048FE4AA001F0E5FD04E0FFF7CAFCE4
:10098000044604B100E0F9E700BF45A001F0DAFD3C
:1009900000204549087048708870C8700871434944
:1009A000087048708870C8700871414908704870B4
:1009B0008870C87008713449887238E10020324963
:1009C000887234E13948407848B93848807830B97D
:1009D0003648C07818B93548007900B927E10020B9
:1009E0002349087028488079324988712648C1799E
:1009F0003048C1712448017A2E4801722248417A58
:100A00002C4841722048807A2A4988720120C87295
:100A10000620087300204873244801782548817314
:100A2000224841782348C1732048817821480174C5
:100A30001E48C1781F4841741C4801791D488174C3
:100A4000162101F069FD322002F0F2F91621194851
:100A500000F0B1F90BA001F075FD002013490870FA
:100A6000487029E099E0DDE0D8E0D3E02BE029E010
:100A700003000020040100200CED00E00000FA0556
:100A8000040000200A000000F80200209402002068
:100A9000C00300202C0000203E0000202000002089
:100AA000303030300A000000390000201B000020E8
:100AB000160000205C0300208870C87008715F4930
:100AC0008872B4E0B3E000205D4908705D480178A9
:100AD000012000F0F1FD00205B4908805BA001F0DF
:100AE00031FD04E0FFF738FD044604B100E0F9E70A
:100AF00000BF56A001F026FD504880795549887105
:100B00004E48C1795348C1714C48017A514801722D
:100B10004A48417A4F4841724848807A4D49887224
:100B20000120C87206200873002048734A480178E3
:100B300048488173484841784648C173464881789F
:100B4000444801744448C17842484174424801799C
:100B500040488174162101F0DFFC322002F068F970
:100B600016213C4800F027F939A001F0EBFC0020E9
:100B70003949087048708870C87008713749087022
:100B800048708870C870087135490870487088705E
:100B9000C87008712949887249E03248407B294968
:100BA000087026488079304988712448C1792E48D8
:100BB000C1712248017A2C4801722048417A2A48A2
:100BC00041721E48807A28498872012048700E219F
:100BD000254801F0A1FC322002F02AF919480078DA
:100BE0002249088001F060FC00201B490870487011
:100BF0008870C87008711949087048708870C8708A
:100C000008711749087048708870C87008710B49DE
:100C100088720CE000200949887208E0002007492A
:100C2000887204E000200549887200E000BF00BF20
:100C300000200F49088000BF56E50000F8020020A0
:100C4000030000202A000020320000203434343415
:100C50000A0000005C030020390000201B00002077
:100C60001600002004010020240400202C05002090
:100C700004000020FA204A49087010204870002023
:100C8000887000214648C1700171417100204449BB
:100C9000887100214248C1710172417200204049AF
:100CA000C87400213E480175FB203D494875FA2073
:100CB0003C49087010204870002088700021394895
:100CC000C170017141710020364988710021354899
:100CD000C171017241720020324981F84B0000213C
:100CE000304880F84C10FB202E4981F84D00FA2046
:100CF0002D490870102048700020887000212A4873
:100D0000C170017141710020274988710021264876
:100D1000C1710172417200202349C872002122482A
:100D20000173FB2020494873FA20204908701020E5
:100D300048700020887000211C48C1700171417109
:100D400000201A49887100211848C171017241724E
:100D500000201649C874002114480175FB2013496E
:100D60004875FA20124908701020487000208870D9
:100D700000210F48C1700171417100200C49887138
:100D800000210B48C1710172417200200849C872EC
:100D9000002107480173FB20054948737047000094
:100DA00094020020F8020020240400205C030020AC
:100DB000C003002070472DE9F04104460E460DE0C7
:100DC0002578281100F030F9074601F0B1FB2846DC
:100DD00000F02AF9074601F0ABFB641C301EA6F1B7
:100DE0000101CEB2ECD1BDE8F081000030B504467F
:100DF00004254FF4302000F06FF80546042D17D17C
:100E00000C48006940F002000A4908610846446144
:100E1000006940F0400008614FF4302000F05CF8B9
:100E200005460448006941F6FD7108400149086122
:100E3000284630BD0020024004200B49C96801F05B
:100E4000010109B101200EE00749C96801F0040160
:100E500009B1022007E00449C96801F0100109B195
:100E6000032000E00420704700200240034800698E
:100E700040F08000014908617047000000200240F6
:100E800070B504460D460426F00200F025F806462B
:100E9000042E11D10948006940F00100074908619A
:100EA0002580F00200F018F806460448006941F673
:100EB000FE71084001490861304670BD00200240C3
:100EC000024803494860034848607047230167456A
:100ED00000200240AB89EFCD00B502460423FFF7A6
:100EE000ABFF034603E0FFF7A7FF0346521E012BAB
:100EF00001D1002AF7D102B90523184600BD2DE91A
:100F0000F04102460025002600200023002400278F
:100F100091F803C00CF00F0591F803C00CF0100C11
:100F2000BCF1000F03D091F802C04CEA050591F81E
:100F300000C0BCF1000F31D0146800202BE04FF04E
:100F4000010C0CFA00F3B1F800C00CEA03069E4253
:100F500020D183004FF00F0C0CFA03F7BC4305FAC5
:100F600003FC4CEA040491F803C0BCF1280F06D13D
:100F70004FF0010C0CFA00FCC2F814C00AE091F822
:100F800003C0BCF1480F05D14FF0010C0CFA00FC76
:100F9000C2F810C0401C0828D1D31460B1F800C0BA
:100FA000BCF1FF0F34DD546800202EE000F1080C86
:100FB0004FF0010808FA0CF3B1F800C00CEA030680
:100FC0009E4221D183004FF00F0C0CFA03F7BC4373
:100FD00005FA03FC4CEA040491F803C0BCF1280FA5
:100FE00005D100F1080C08FA0CF8C2F8148091F849
:100FF00003C0BCF1480F07D100F1080C4FF0010805
:1010000008FA0CF8C2F81080401C0828CED35460AF
:10101000BDE8F081416170470161704701460A886F
:1010200090B2704700BFFEE70146002001F00F02BA
:10103000092A04DC01F00F0202F1300003E001F0A4
:101040000F023732D0B270474CF6CC4001490860ED
:10105000704700000030004010B500F013F810BDDC
:1010600070B505460C4645F2555000F01FF828466D
:1010700000F010F8204600F013F800F003F8FFF736
:10108000E3FF70BD4AF6AA200149086070470000DE
:1010900000300040014948607047000000300040C7
:1010A0000149886070470000003000400149086035
:1010B000704700000030004000BFFEE770470000AE
:1010C0007CB5054612A103C9CDE9000108212846D7
:1010D00001F0B8F905236A463021284600F0BAFE2F
:1010E00005236A461021284600F024FE002406E06D
:1010F0001DF80400A52800D003E0601CC4B2052C34
:10110000F6DB00BF052C01D001207CBD0020FCE7F0
:10111000A5A5A5A5A500000008B501211C2000F08B
:101120009BFF4020ADF8000010208DF80300032045
:101130008DF8020069463248FFF7E1FE4021304851
:10114000FFF76AFF1020ADF8000069462D48FFF751
:10115000D6FE10212B48FFF75FFF8020ADF800007E
:1011600048208DF8030003208DF8020069462448CA
:10117000FFF7C5FE4FF40070ADF8000010208DF8A9
:10118000030003208DF8020069461D48FFF7B7FEF3
:101190004FF400711A48FFF73FFF4FF48050ADF84D
:1011A000000069461648FFF7AAFE4FF48051144824
:1011B000FFF732FF4FF48070ADF8000048208DF843
:1011C000030003208DF8020069460D48FFF797FEE3
:1011D00001F066F801F022F800200B4908600120B8
:1011E0000A49C1F89001002007490C31086001202C
:1011F0000749C1F8B0010821002001F023F908BD1A
:10120000000C014000080140988121420000214269
:101210000080214210B5044602222321204600F01E
:1012200057FE05231E4A2A21204600F013FE0523FF
:101230001B4A3021204600F00DFE3022212120469D
:1012400000F046FE01222221204600F041FE1A2233
:101250002521204600F03CFE24222621204600F0D5
:1012600037FE0F222021204600F032FE0A223121D3
:10127000204600F02DFE01223D21204600F028FEF0
:1012800000223C21204600F023FE70222721204628
:1012900000F01EFEFF22E221204600F019FE10BDE4
:1012A000B131000810B5044602222321204600F087
:1012B0000FFE04231E4A2A21204600F0CBFD042302
:1012C0001B4A3021204600F0C5FD30222121204656
:1012D00000F0FEFD01222221204600F0F9FD12223D
:1012E0002521204600F0F4FD24222621204600F08E
:1012F000EFFD0F222021204600F0EAFD08223121D7
:10130000204600F0E5FD01223D21204600F0E0FDF1
:1013100000223C21204600F0DBFD702227212046E0
:1013200000F0D6FDFF22E221204600F0D1FD10BDE5
:10133000E831000810B5044602222321204600F0BF
:10134000C7FD04231E4A2A21204600F083FD042302
:101350001B4A3021204600F07DFD3022212120460D
:1013600000F0B6FD01222221204600F0B1FD282226
:101370002521204600F0ACFD0C222621204600F05D
:10138000A7FD0F222021204600F0A2FD06223121D8
:10139000204600F09DFD01223D21204600F098FDF1
:1013A00000223C21204600F093FD70222721204698
:1013B00000F08EFDFF22E221204600F089FD10BDE5
:1013C000DE31000810B5044602222321204600F039
:1013D0007FFD04231E4A2A21204600F03BFD042302
:1013E0001B4A3021204600F035FD302221212046C5
:1013F00000F06EFD01222221204600F069FD33221B
:101400002521204600F064FD04222621204600F01C
:101410005FFD0F222021204600F05AFD09223121D4
:10142000204600F055FD01223D21204600F050FDF0
:1014300000223C21204600F04BFD7022272120464F
:1014400000F046FDFF22E221204600F041FD10BDE4
:10145000D431000810B5044602222321204600F0B2
:1014600037FD05231E4A2A21204600F0F3FC052300
:101470001B4A3021204600F0EDFC3F22212120466E
:1014800000F026FD01222221204600F021FD12223B
:101490002521204600F01CFD04222621204600F0D4
:1014A00017FD0F222021204600F012FD0A223121D3
:1014B000204600F00DFD01223D21204600F008FDF0
:1014C00000223C21204600F003FD70222721204607
:1014D00000F0FEFCFF22E221204600F0F9FC10BDE6
:1014E000A231000810B5044602222321204600F054
:1014F000EFFC05231E4A2A21204600F0ABFC052301
:101500001B4A3021204600F0A5FC30222121204634
:1015100000F0DEFC01222221204600F0D9FC12223C
:101520002521204600F0D4FC21222621204600F06F
:10153000CFFC0F222021204600F0CAFC0A223121D4
:10154000204600F0C5FC00223D21204600F0C0FCF2
:1015500001223C21204600F0BBFC702227212046BE
:1015600000F0B6FCFF22E221204600F0B1FC10BDE5
:101570009331000810B5044601222321204600F0D3
:10158000A7FC05231E4A2A21204600F063FC052300
:101590001B4A3021204600F05DFC302221212046EC
:1015A00000F096FC01222221204600F091FC192235
:1015B0002521204600F08CFC04222621204600F044
:1015C00087FC0F222021204600F082FC06223121D8
:1015D000204600F07DFC01223D21204600F078FCF1
:1015E00000223C21204600F073FC70222721204677
:1015F00000F06EFCFF22E221204600F069FC10BDE5
:10160000C031000810B504461CB900202749086005
:1016100003E0002025490C310860012223212046E7
:1016200000F056FC0323224A2A21204600F012FC37
:101630000323204A3021204600F00CFC0122212106
:10164000204600F045FC01222221204600F040FC0B
:101650002A222521204600F03BFC04222621204698
:1016600000F036FC0F222021204600F031FC06223B
:101670003D21204600F02CFC01223C21204600F0B8
:1016800027FC70222721204600F022FCFF22E221C5
:10169000204600F01DFC1CB901200449086003E04D
:1016A000012002490C31086010BD000098812142E0
:1016B000893100088431000870B504460D461CB914
:1016C00000203349086003E0002031490C310860F4
:1016D000122D52D2DFE805F0090D1115191D212533
:1016E000292D3135393D4145494D2046FFF7FAFE58
:1016F00043E0204600F046FA3FE0204600F0D2FAF0
:101700003BE02046FFF7A6FE37E0204600F0AAF9AE
:1017100033E0204600F0CEF82FE02046FFF77AFDB8
:101720002BE0204600F056F927E0204600F072FA40
:1017300023E02046FFF71EFF1FE0204600F02AF8B6
:101740001BE0204600F0D6F917E0204600F06AF8CA
:1017500013E02046FFF736FE0FE02046FFF70AFFB2
:101760000BE02046FFF7E6FD07E0204600F0EAF830
:1017700003E02046FFF796FD00BF00BF1CB9012023
:101780000349086003E0012001490C31086070BD85
:101790009881214210B5044602222321204600F000
:1017A00097FB04231E4A2A21204600F053FB042302
:1017B0001B4A3021204600F04DFB302221212046DB
:1017C00000F086FB01222221204600F081FB20222E
:1017D0002521204600F07CFB20222621204600F017
:1017E00077FB0F222021204600F072FB08223121D6
:1017F000204600F06DFB01223D21204600F068FBF1
:1018000000223C21204600F063FB70222721204665
:1018100000F05EFBFF22E221204600F059FB10BDE4
:10182000C531000810B5044602222321204600F0ED
:101830004FFB04231E4A2A21204600F00BFB042301
:101840001B4A3021204600F005FB30222121204692
:1018500000F03EFB01222221204600F039FB12223B
:101860002521204600F034FB24222621204600F0CA
:101870002FFB0F222021204600F02AFB0A223121D3
:10188000204600F025FB01223D21204600F020FBF0
:1018900000223C21204600F01BFB7022272120461D
:1018A00000F016FBFF22E221204600F011FB10BDE4
:1018B000CF31000810B5044602222321204600F053
:1018C00007FB05231E4A2A21204600F0C3FA052300
:1018D0001B4A3021204600F0BDFA3022212120464B
:1018E00000F0F6FA01222221204600F0F1FA12223D
:1018F0002521204600F0ECFA24222621204600F083
:10190000E7FA0F222021204600F0E2FA0A223121D4
:10191000204600F0DDFA01223D21204600F0D8FAF1
:1019200000223C21204600F0D3FA702227212046D5
:1019300000F0CEFAFF22E221204600F0C9FA10BDE5
:10194000AC31000810B5044602222321204600F0E5
:10195000BFFA04231E4A2A21204600F07BFA042302
:101960001B4A3021204600F075FA30222121204602
:1019700000F0AEFA01222221204600F0A9FA12223C
:101980002521204600F0A4FA24222621204600F03A
:101990009FFA0F222021204600F09AFA08223121D6
:1019A000204600F095FA01223D21204600F090FAF1
:1019B00000223C21204600F08BFA7022272120468D
:1019C00000F086FAFF22E221204600F081FA10BDE5
:1019D000E331000810B5044601222321204600F01F
:1019E00077FA05231E4A2A21204600F033FA052300
:1019F0001B4A3021204600F02DFA302221212046BA
:101A000000F066FA01222221204600F061FA10223D
:101A10002521204600F05CFA04222621204600F011
:101A200057FA0F222021204600F052FA06223121D7
:101A3000204600F04DFA01223D21204600F048FAF0
:101A400000223C21204600F043FA70222721204644
:101A500000F03EFAFF22E221204600F039FA10BDE4
:101A6000B631000810B5044602222321204600F0BA
:101A70002FFA05231E4A2A21204600F0EBF9052300
:101A80001B4A3021204600F0E5F930222121204672
:101A900000F01EFA01222221204600F019FA12223B
:101AA0002521204600F014FA24222621204600F0A9
:101AB0000FFA0F222021204600F00AFA08223121D5
:101AC000204600F005FA01223D21204600F000FAF0
:101AD00000223C21204600F0FBF9702227212046FD
:101AE00000F0F6F9FF22E221204600F0F1F910BDE6
:101AF000A731000810B5044602222321204600F039
:101B0000E7F904231E4A2A21204600F0A3F9042302
:101B10001B4A3021204600F09DF930222121204629
:101B200000F0D6F901222221204600F0D1F91C2232
:101B30002521204600F0CCF924222621204600F061
:101B4000C7F90F222021204600F0C2F908223121D6
:101B5000204600F0BDF901223D21204600F0B8F9F1
:101B600000223C21204600F0B3F9702227212046B4
:101B700000F0AEF9FF22E221204600F0A9F910BDE5
:101B8000CA31000810B5044603222321204600F084
:101B90009FF905231E4A2A21204600F05BF9052300
:101BA0001B4A3021204600F055F93F2221212046D2
:101BB00000F08EF93F222221204600F089F92822E8
:101BC0002521204600F084F904222621204600F039
:101BD0007FF90B222021204600F07AF90A223121D8
:101BE000204600F075F901223D21204600F070F9F1
:101BF00000223C21204600F06BF97022272120466C
:101C000000F066F9FF22E221204600F061F910BDE4
:101C10009831000810B5044601222321204600F027
:101C200057F903231E4A2A21204600F013F9032303
:101C30001B4A3021204600F00DF930222121204698
:101C400000F046F901222221204600F041F92A2223
:101C50002521204600F03CF904222621204600F0F0
:101C600037F90F222021204600F032F907223121D6
:101C7000204600F02DF900223D21204600F028F9F1
:101C800001223C21204600F023F970222721204622
:101C900000F01EF9FF22E221204600F019F910BDE4
:101CA000BB31000810B5044603222321204600F072
:101CB0000FF905231E4A2A21204600F0CBF8052300
:101CC0001B4A3021204600F0C5F830222121204651
:101CD00000F0FEF801222221204600F0F9F810223F
:101CE0002521204600F0F4F804222621204600F0A9
:101CF000EFF80F222021204600F0EAF80A223121D5
:101D0000204600F0E5F801223D21204600F0E0F8F1
:101D100000223C21204600F0DBF8702227212046DB
:101D200000F0D6F8FF22E221204600F0D1F810BDE5
:101D30009D3100082DE9F0478046894615461E462C
:101D4000B8F1000F16D100201749086049464046F7
:101D500000F024FB0746002406E0FF21404600F087
:101D60001DFB2855601CC4B2B442F6DB01200E49AD
:101D7000086015E000200D4908604946404600F023
:101D80000DFB0746002406E0FF21404600F006FB5D
:101D90002855601CC4B2B442F6DB01200349086038
:101DA0003846BDE8F087000090012142B081214211
:101DB00070B505460E4685B90020114908603146C8
:101DC000284600F0EBFAFF21284600F0E7FA044627
:101DD00001200C49C1F890010FE000200A49086079
:101DE0003146284600F0DAFAFF21284600F0D6FAFC
:101DF000044601200549C1F8B001204670BD00002D
:101E00009001214200002142B08121420080214204
:101E100070B506460D461021304600F013FB072131
:101E20003046FFF7C5FF044622462721304600F022
:101E30004FF804F0400050B10A232A466121304691
:101E4000FFF778FFFF22E221304600F041F82046FC
:101E500070BD00002DE9F0478046894615461E46B4
:101E6000B8F1000F16D100201749086049464046D6
:101E700000F094FA0746002406E015F8011B4046DE
:101E800000F08CFA601CC4B2B442F6DB01200E49AB
:101E9000086015E000200D4908604946404600F002
:101EA0007DFA0746002406E015F8011B404600F0C5
:101EB00075FA601CC4B2B442F6DB01200349086025
:101EC0003846BDE8F087000090012142B0812142F0
:101ED0002DE9F04104460E46154684B9002011490B
:101EE00008603146204600F059FA07462946204648
:101EF00000F054FA01200C49C1F890010FE00020D5
:101F00000A4908603146204600F048FA074629464B
:101F1000204600F043FA01200549C1F8B0013846D7
:101F2000BDE8F0819001214200002142B0812142B0
:101F30000080214208B54FF4C06000F071F82620FF
:101F40008DF8000001208DF8010002208DF80200BC
:101F500001208DF80300684600F02AF827208DF84C
:101F6000000001208DF801008DF802008DF80300BB
:101F7000684600F01DF825208DF8000000208DF83F
:101F8000010001208DF802008DF80300684600F082
:101F90000FF81D208DF8000000208DF801008DF84D
:101FA000020001208DF80300684600F001F808BD2A
:101FB00070B5002100230F22C47804B3154C2468A7
:101FC00004F4E064C4F5E064210AC1F10403CA40EA
:101FD000447804FA03F184781440214309010E4C3B
:101FE0000678A155047804F01F050124AC4005785B
:101FF0006D11AD0005F1E025C5F8004109E0047858
:1020000004F01F050124AC40044D0678761145F814
:10201000264070BD0CED00E000E400E080E100E04F
:1020200002490143024A1160704700000000FA05AE
:102030000CED00E07047000029B1064AD269024366
:10204000044BDA6104E0034AD2698243014BDA614E
:10205000704700000010024029B1064A926902430D
:10206000044B9A6104E0034A92698243014B9A61EE
:10207000704700000010024070B5012144F20D00CD
:10208000FFF7EAFF01210220FFF7D6FF042000F04E
:1020900013FB1249B1F1807F00D31DE021F07F4096
:1020A000401E4FF0E022506150170F22002807DA3F
:1020B00013071D0E0A4B00F00F04241F1D5503E0EB
:1020C00013071C0E074B1C5400BF00204FF0E022EA
:1020D00090610720106100BF70BD000080A903005F
:1020E00018ED00E000E400E070B5002100230024BA
:1020F000002200252C4E766806F00C0121B104293F
:1021000005D0082921D105E0284E066020E0274EA1
:1021100006601DE0244E766806F47013224E766841
:1021200006F48034022606EB93431CB9204E5E432E
:10213000066009E01C4E7668C6F34046751C1B4ECF
:10214000B6FBF5F65E43066002E0184E066000BF7F
:1021500000BF154E766806F0F0010909154E725C55
:102160000668D6404660104E766806F4E061090ABB
:10217000104E725C4668D64086600B4E766806F458
:102180006051C90A0B4E725C4668D640C660064E66
:10219000766806F44041890B074E725CC668B6FB50
:1021A000F2F6066170BD00000010024000127A00D5
:1021B00000093D00880000209800002010B586B07E
:1021C0000024142101A8FDF7D6FF0A2201A908481E
:1021D00000F012F800BF07E001A810F81400054A4B
:1021E00002F81400601CC4B20A2CF5DB06B010BD66
:1021F000000003084005002070B504460D46164651
:10220000002300BF07E02046FEF708FF25F8130073
:10221000A41C581CC3B2B342F5DB70BD00B587B037
:10222000012141F20500FFF717FFE020ADF818008B
:1022300018208DF81B0003208DF81A0006A91648F7
:10224000FEF75DFEE0211448FEF7E6FE0020ADF843
:1022500004004FF48270ADF806000020ADF80800CD
:10226000ADF80A00ADF80C004FF40070ADF80E00A8
:102270001820ADF810000020ADF812000720ADF8CE
:10228000140001A9054800F06BF80121034800F093
:102290004DF807B000BD00000008014000300140CB
:1022A00000B587B001218803FFF7C6FE0121092090
:1022B000FFF7D2FE4FF46040ADF8180018208DF8FB
:1022C0001B0003208DF81A0006A91648FEF717FE1A
:1022D0004FF460411348FEF79FFE0020ADF8040064
:1022E0004FF48270ADF806000020ADF80800ADF89C
:1022F0000A00ADF80C004FF40070ADF80E00182085
:10230000ADF810000020ADF812000720ADF8140061
:1023100001A9054800F024F80121034800F006F85F
:1023200007B000BD000C01400038004021B1028818
:1023300042F04002028004E002884FF6BF731A4068
:10234000028070470246002013890B400BB1012028
:1023500000E00020704701468889704781817047FE
:1023600010B50022028802F441520B884C882343A6
:102370008C882343CC8823430C8923434C892343F3
:102380008C892343CC8923431A430280838B4FF2E9
:10239000FF74234083830B8A038210BD2DE9F04133
:1023A00006460F4626BB06E0601CC4B2C82C02DB02
:1023B0000020BDE8F08102212048FFF7C3FF00287C
:1023C000F2D039461D48FFF7C9FF002405E0601C24
:1023D000C4B2C82C01DB0020EBE701211748FFF74E
:1023E000B1FF0028F3D01548FFF7B5FFC5B222E0D2
:1023F00005E0601CC4B2C82C01DB0020D9E7022133
:102400000F48FFF79FFF0028F3D039460C48FFF72D
:10241000A5FF002405E0601CC4B2C82C01DB00202D
:10242000C7E701210648FFF78DFF0028F3D00448D5
:10243000FFF791FFC5B22846BBE70000003001401E
:102440000038004070B505460C467DB90F4800883D
:102450004FF6C77108400D490880084600882043A0
:10246000088001210A48FFF761FF0EE00848008854
:102470004FF6C77108400649088008460088204387
:10248000088001210248FFF751FF70BD0030014074
:1024900000380040704770B504460D462946204676
:1024A000FEF7EEFC70BD000010B586B000241421CC
:1024B00001A8FDF760FE00BF07E00B4830F81400EC
:1024C00001A921F81400601CC4B20A2CF5DB0748EE
:1024D00000F0EAF80A2201A9044800F009F800F027
:1024E0007AFC06B010BD00002C0500200000030897
:1024F0002DE9F04105460F461646002400BF07E0CF
:1025000037F814102846FFF7C6FFAD1C601CC4B294
:10251000B442F5DBBDE8F08170B504460D46034AD0
:102520002946204600F028F870BD00000038014020
:1025300010B504460249204600F00EF810BD000018
:102540000044004010B504460249204600F02DF832
:1025500010BD00000044004070B504460D4600BFA9
:102560008021284600F064FB0028F9D02146284647
:1025700000F02BFC012070BD2DE9F04104460D4612
:10258000164614B90120BDE8F0810AE014F8017B79
:1025900031463846FFF7E0FF08B90020F3E7681E30
:1025A00085B2002DF2D10120EDE770B504460E464C
:1025B0000CB9012070BD11E014F8015B0A2D06D1A1
:1025C00031460D20FFF7C8FF08B90020F2E7314679
:1025D0002846FFF7C1FF08B90020EBE72078002864
:1025E000EAD10120E6E710B500F002F810BD0000C6
:1025F0000CB50020019000902A48006840F480301B
:102600002849086000BF2748006800F400300090A7
:102610000198401C0190009818B90198B0F5A06F7E
:10262000F1D12048006800F4003010B10120009082
:1026300001E0002000900098012831D1194840683D
:102640001849486008464068486008464068486045
:102650000846406820F47C1048600846406840F412
:10266000981048600846006840F08070086000BF1D
:102670000C48006800F000700028F9D00948406854
:1026800020F00300074948600846406840F0020017
:10269000486000BF0348406800F00C000828F9D1EA
:1026A0000CBD00000010024010B50446FEF708FC07
:1026B0002046FEF79BFB10BD042808D14FF0E02117
:1026C000096941F004014FF0E022116107E04FF089
:1026D000E021096921F004014FF0E0221161704707
:1026E0007047000010B51448006840F0010012491E
:1026F000086008464068114908400F49486008468C
:1027000000680F4908400C4908600846006820F43A
:10271000802008600846406820F4FE0048604FF4BE
:102720001F0088600020C862FFF75DFF4FF0006067
:102730000449086010BD0000001002400000FFF8CE
:10274000FFFFF6FE08ED00E010B50121204800F083
:102750007EF800283AD001211D4800F069F81D4894
:102760000088401C1B4908801B480088401C1A49EF
:1027700008801A480088401C1849088018480078CA
:10278000C0B14FF400711748FEF746FC16480088A8
:10279000401C1549088008460088B0F5C87F09DB51
:1027A0004FF400710F48FEF735FC00200E490880F9
:1027B0000B4908700948008841F28831884202D1EB
:1027C00000200649088001200849087010BD00005B
:1027D00000040040200000203200002022000020E1
:1027E00025000020001001402600002024000020C9
:1027F0003EB505460C4601210220FFF71DFCADF851
:102800000450ADF800400020ADF80600ADF802001D
:102810006946064800F036F801221146034800F0E8
:1028200027F80121014800F006F83EBD00040040F1
:10283000CA430282704721B1028842F0010202803D
:1028400004E002884FF6FE731A400280704730B5EC
:102850000246002000230024158A05EA0103958919
:1028600005EA010413B10CB1012000E0002030BDE5
:102870001AB183890B43838102E083898B4383816F
:1028800070470000002202881D4B98420ED01D4B5D
:1028900098420BD0B0F1804F08D01B4B984205D026
:1028A0001A4B984202D01A4B984204D14FF68F73BC
:1028B0001A404B881A43174B984207D0164B984240
:1028C00004D04FF6FF431A40CB881A4302808B880E
:1028D00083850B8803850A4B98420BD0094B98429D
:1028E00008D00E4B984205D00D4B984202D00D4BAC
:1028F000984201D10B7A038601238382704700003E
:10290000002C014000340140000400400008004059
:10291000000C004000100040001400400040014046
:10292000004401400048014010B540F225511248D2
:1029300000F08BF988B140F225510F4800F0CFF834
:102940000D4800F03DFAC4B20C480D4909784454D2
:102950000B480078401C0A4908700821064800F01E
:1029600067F9012806D10821034800F0AFF80248B2
:1029700000F026FA10BD00000038014004010020DC
:102980000300002010B540F22551124800F05DF917
:1029900088B140F225510F4800F0A1F80D4800F031
:1029A0000FFAC4B20C480D49097844540B4800781A
:1029B000401C0A4908700821064800F039F901282E
:1029C00006D10821034800F081F8024800F0F8F928
:1029D00010BD000000440040EC04002085000020F1
:1029E00010B586B0044601210520FFF735FB012113
:1029F0004804FFF721FB0420ADF8140003208DF8F4
:102A0000160018208DF8170005A91548FEF777FA6B
:102A10000820ADF8140004208DF8170005A910480F
:102A2000FEF76DFA01940020ADF80800ADF80A0039
:102A3000ADF80C00ADF810000C20ADF80E0001A9A7
:102A4000084800F051F9012240F22551054800F0F4
:102A500026F90121034800F051F806B010BD00002E
:102A6000000801400044004010B540F225511448D0
:102A700000F0EBF8B0B140F22551114800F02FF80A
:102A80000F4800F09DF9C4B20E480F49097844542C
:102A90000D480078401C0C4908700846007800F08A
:102AA0000F0008700821064800F0C2F8012806D17E
:102AB0000821034800F00AF8014800F081F910BD30
:102AC00000480040CC0100200900002001F4007201
:102AD000B2F5007F00D100BFCA430280704710B535
:102AE0000022002340F66A14A14200D100BF0A125E
:102AF00001249440A3B2DC43048010BD21B182893B
:102B000042F40052828104E082894DF6FF731A403C
:102B10008281704700B585B0012144F20400FFF7BF
:102B20009BFA4FF40070ADF8000003208DF802000E
:102B300018208DF8030069463948FEF7E0F94FF494
:102B40008060ADF8000004208DF803006946344829
:102B5000FEF7D5F94FF4164001900020ADF80800BB
:102B6000ADF80A00ADF80C00ADF810000C20ADF87F
:102B70000E0001A92B4800F0B7F8012240F22551C0
:102B8000284800F08CF801212648FFF7B7FF012103
:102B90008804FFF751FA01210820FFF75DFA4FF48E
:102BA0008060ADF8000003208DF8020018208DF839
:102BB000030069461C48FEF7A2F94FF40060ADF827
:102BC000000004208DF8030069461748FEF797F9C6
:102BD0004FF4965001900020ADF80800ADF80A00BF
:102BE000ADF80C00ADF810000C20ADF80E0001A9F6
:102BF0000E4800F079F801A90C4800F075F80122A0
:102C000040F22551094800F04AF801210748FFF732
:102C100075FF40210348FFF759FF05B000BD0000D4
:102C20000008014000380140000C0140004800400D
:102C300002460020B1F5007F00D100BF13880B4091
:102C40000BB1012000E00020704770B5024600245F
:102C500000230025002040F66A16B14200D100BFD3
:102C6000C1F3421501F01F03012606FA03F3012DFB
:102C700002D19689334006E0022D02D1168A3340F4
:102C800001E0968A33400C12012606FA04F41688F5
:102C9000344013B10CB1012000E0002070BDF0B54C
:102CA0000346002400260025002040F66A17B9429A
:102CB00000D100BF1846C1F3421401F01F060127DE
:102CC00007FA06F5012C01D10C3004E0022C01D1E9
:102CD000103000E014301AB107682F43076002E09B
:102CE0000768AF430760F0BD2DE9F04786B00546A1
:102CF0000E460024A24600BFA1460027B08900B1BD
:102D000000BF2F462C8A4CF6FF700440F088044325
:102D10002C82AC894EF6F3100440B0883189084308
:102D2000718908430443AC81AC8A4FF6FF400440EC
:102D3000B0890443AC8201A8FFF7D6F91F48874247
:102D400002D1DDF810A001E0DDF80CA0A88900F4A4
:102D5000004040B10AEBCA0000EB0A10316849009C
:102D6000B0FBF1F807E00AEBCA0000EB0A1031688B
:102D70008900B0FBF1F86420B8FBF0F004012009F1
:102D8000642101FB1089A88900F4004040B1322081
:102D900000EBC900B0FBF1F000F00700044308E0CD
:102DA000322000EB09106421B0FBF1F000F00F00BD
:102DB00004432C8106B0BDE8F087000000380140D4
:102DC00001468888C0F308007047C1F3080282807A
:102DD000704700BFFEE710B5FEF748F810BD0000D1
:102DE000014A024900F013B85D2E00089C00002043
:102DF00002E008C8121F08C1002AFAD170477047C4
:102E0000002001E001C1121F002AFBD170472DE90B
:102E1000F04116460F460446002503E03946B04708
:102E2000641C6D1C20780028F8D12846BDE8F0818C
:102E300010B502460BE0C82007E0122101E04B1E4E
:102E400099B20029FBDC431E98B20028F5DC131E62
:102E5000A2F10104A2B2EED110BD000070B504468B
:102E60000D46E0B20549088000BF40210348001F1D
:102E7000FFF7DEFE0028F8D0204670BD0438014080
:102E800008B501211020FFF7E7F80120ADF8000098
:102E900010208DF8030003208DF8020069460D48CC
:102EA000FEF72DF801210B48FEF7B6F84FF400703D
:102EB000ADF8000010208DF8030003208DF802000B
:102EC00069460448FEF71BF84FF400710148FEF70D
:102ED000A1F808BD00100140FFF7CEF8FFF72AF86F
:102EE00040F271210420FEF7BBF8FEF7B5F841F679
:102EF0001F410920FFF77CFCFFF7C2FFFFF70AFE26
:102F00004FF4E130FFF76CFDFEF706F9FEF7A4F889
:102F100002E049A0FFF764FF0120FEF7D1F8002886
:102F2000F7D1FDF7A7FEFEF797F847480068C043C2
:102F30004649C1F88001C820FFF77AFF4348D0F81E
:102F40008001C0434149C1F88001062140A0FDF73E
:102F500032FF41A0FFF7F6FAFEF77EF83FA0FFF739
:102F60003FFF0120FEF74EFBFFF728F944480078A9
:102F70004449087008460078122852D2DFE800F071
:102F8000090D1115191D2125292D3135393D4145D1
:102F9000494D3DA0FFF724FF43E03EA0FFF720FF8F
:102FA0003FE03FA0FFF71CFF3BE040A0FFF718FF0A
:102FB00037E041A0FFF714FF33E042A0FFF710FF16
:102FC0002FE044A0FFF70CFF2BE045A0FFF708FF20
:102FD00027E046A0FFF704FF23E047A0FFF700FF2C
:102FE0001FE048A0FFF7FCFE1BE049A0FFF7F8FE3A
:102FF00017E04BA0FFF7F4FE13E04EA0FFF7F0FE42
:103000000FE050A0FFF7ECFE0BE052A0FFF7E8FE48
:1030100007E054A0FFF7E4FE03E056A0FFF7E0FE50
:1030200000BF00BF3220FFF703FF03E0FDF7D4F835
:10303000FDF71EFBFAE7000054686520322E344786
:10304000204572726F7221008001224200002242EC
:1030500031323334353600000A0000000A5043B6DE
:10306000D4C2EBC8EDBCFECDA8D3C3B0E6B1BE560A
:10307000312E382D32303138303530340A000000EE
:10308000400500202A000020BDADCEF7D0ADD2E92A
:103090000D0A0000CCECB2A8D0ADD2E90D0A0000B8
:1030A000D4C6C4CFD0ADD2E90D0A0000B9F3D6DD45
:1030B000D0ADD2E90D0A0000CBC4B4A8D0ADD2E99E
:1030C0000D0A0000C4DAC3C9B9C5D0ADD2E90D0AF2
:1030D00000000000B0B2BBD5D0ADD2E90D0A0000AF
:1030E000C9BDCEF7D0ADD2E90D0A000056434F4D11
:1030F000B2E2CAD40D0A0000C1C9C4FEB5E7D0C50A
:103100000D0A0000C1C9C4FED2C6B6AF0D0A000048
:103110005470D7A8D3C3D0ADD2E90D0A0000000087
:10312000C4DAC3C9B9C5D2C6B6AFD0ADD2E90D0AAB
:1031300000000000B9E3CEF7D2C6B6AFD0ADD2E9F9
:103140000D0A0000CBC4B4A8B5E7D0C5D0ADD2E914
:103150000D0A0000B8A3BDA8D5E6D7C6D0ADD2E908
:103160000D0A0000CBD5D6DDC4BEC0BCD0ADD2E9BF
:103170000D0A0000D6D8C7ECD2C6B6AFD0ADD2E9A2
:103180000D0A0000344310100134431010013320A5
:103190000D547933200D547934431010010110106F
:1031A00043343223ABBA013412BBAA013412867500
:1031B000014656431000346E46100134431010018E
:1031C000862C95010136E4A7BC014218BAE8013407
:1031D0001286750133200D5400862C9500005A4547
:1031E0004E4B00AABB1234003412BBAA00000000F0
:1031F0001032000800000020A0000000F02D0008A0
:10320000B0320008A0000020605F0000002E00081F
:10321000000000000000000000000000D1D1E0D05C
:1032200000000000D2D200000000000000000000FA
:10323000000000000000000000000000000000008E
:10324000000000000000000000000000000000007E
:103250000000313233343536373839313233343592
:103260003637383900000000000000000000000080
:103270000000313233343536373839313233343572
:103280003637383900000000000000000000000060
:103290000000000000000000000000000102030424
:1032A00001020304060708090204060800000000E2
:0400000508000131BD
:00000001FF
